:10000000000002308A00FC2A8030A100FE30E92086
:100010000130E9207530A90030305429A101A11721
:10002000B700FE30E9203708E928C900BA1F1A28AE
:100030002D30E920BC0F2128BB0F2128BA0A031953
:10004000BA0AC101C201C301C401BA176A30B907B3
:100050000310BA0CBB0CBC0CC40CC30CC20CC10CFE
:10006000B90F28283C083902BC07B9023B083A02FC
:10007000BB07BA02A50174202E30E920CA01031083
:10008000410DBC00420DBB00430DBA00440DB90048
:10009000CA0D0310BC0DBB0DBA0DB90DCA0D410838
:1000A000BC0742080318420FBB0743080318430F5D
:1000B000BA0744080318440FB9070318CA0F0310FE
:1000C000BC0DBB0DBA0DB90DCA0D4A08303EE92072
:1000D0003C08C1003B08C2003A08C3003908C4000C
:1000E000C90B3E280310E229A0112508031D7B2817
:1000F000A0150A30A5003C08AB003B08AA003A084E
:10010000A9003908A800A401B301B201B1010A3065
:10011000B0006821A40A24082502031D84283008A1
:10012000031DA011A01D9628250B99283008303EEC
:10013000E920A50B7B28E229B5008611061183165C
:10014000861106110F30860583123508A018C628BF
:100150003E30A900803054213330B400DA2013300F
:10016000A90088305421DA2064305321DA20643029
:1001700053212230B400DA202830C5200C30C520AD
:100180000630C520A0143508C6282014B400201C51
:10019000D4280611033C031CD928D9200130A9001A
:1001A000F4305421031408002014FE3C0319E728FE
:1001B0000615201C201086150F3086053408F039EE
:1001C00086048611B40E2018DA28323053213508FF
:1001D000E229A11B9C280800AC0008302719013037
:1001E000AD00AC0C230884002608FF3A8005841774
:1001F00080052608031880043C305321260880041B
:10020000AD0BF1280314E229083027190130AD00A5
:10021000AC01230884002608FF3A80058417800576
:100220002608800484130005FF3E271DAC0C271907
:10023000AC0D32305321AD0B0B292C080314E229ED
:10024000A71CE2292629A700271CE22923088400ED
:100250002608FF3A8005841780050130A900F43094
:100260005421260880040130A900F4305429A40048
:10027000A201240803178D000313250803178F001C
:100280004A210319E229E920A40A0319A50AA20FA9
:100290003929E229831603178C170C14000000007B
:1002A00083120C08E229A901E83EA800A909FC3044
:1002B000031C5D29A80703185A29A8070000A90FE5
:1002C0005A2928186329A81C6729000067290800F3
:1002D0002B0833068039B500AB1F7929A809A90975
:1002E000AA09AB09A80A0319A90A0319AA0A03193A
:1002F000AB0AB31F8629B009B109B209B309B00A24
:100300000319B10A0319B20A0319B30AAC01AD010A
:10031000AE01AF01BD01BE01BF01C001330832040F
:10032000310430040319C4292030B4000310A80D8F
:10033000A90DAA0DAB0DBD0DBE0DBF0DC00D33082F
:100340004002031DAD2932083F02031DAD293108CB
:100350003E02031DAD2930083D02031CBE293008B2
:10036000BD023108031C310FBE023208031C320FDC
:10037000BF023308031C330FC0020314AC0DAD0DD4
:10038000AE0DAF0DB40B9629B51FD129AC09AD093F
:10039000AE09AF09AC0A0319AD0A0319AE0A031975
:1003A000AF0A3D08B0003E08B1003F08B200400867
:1003B000B3002C08A8002D08A9002E08AA002F08B9
:1003C000AB00E22983138312031308008030C606B2
:1003D00045084102C9000318072AC909C90A41088A
:1003E000CC004508C1004C08C5004208CC004608B6
:1003F000C2004C08C6004308CC004708C3004C08A4
:10040000C7004408CC004808C4004C08C8001A3093
:1004100049020318E229C5080319E229BD0142086F
:10042000CC004606CD00C217C6170830C902031C0F
:10043000212A4808BD004708C8004608C700C60171
:10044000152AC90703192D2A0310C60CC70CC80C9E
:10045000BD0CC903C908031D242ACD1F762A4808EC
:10046000C4024708031C470FC3024608031C460F7B
:10047000C2020318452AC209C309C409C40F432A8A
:10048000C30A0319C20A8030CC06BD09BD0A03198C
:10049000502AC403440F502AC303430A0319C2035A
:1004A0000430C900C208031D642A4308C20044087E
:1004B000C3003D08C400BD010830C102031C972AD7
:1004C000C9030319972A522AC21B6F2A0310BD0DB4
:1004D000C40DC30DC20DC1030319972A642A4B1F13
:1004E000752ABD1F752ABD018D2A962A4808C407A2
:1004F00047080318470FC30746080318460FC207EB
:10050000031C892AC20CC30CC40CBD0CC10A0319FC
:10051000992A4B1F962ABD1F962AC40F962AC30FED
:10052000962AC20F962A03144110822AA02AC101DA
:100530009C2ACB16FF30C100C401C3018030C20029
:10054000CC1BA32AC213E229C301C4019630CC00FC
:10055000CD13C41FB72AC409C309C209C109C10FF9
:10056000B62AC20FB62AC30A0319C40ACD17C40893
:100570000319D22A4B1FC92AC41FC92AC20FC92A6C
:10058000C30FC92AC40FC92A0314C40CC30CC20C5C
:10059000CC0A0830CC074208C1004308C200440816
:1005A000C300E72AC308031DE72A0830CC0242082B
:1005B000031DE32A0830CC024108031DE22A440847
:1005C000CC00F12AC101C3004108C200C101C31B14
:1005D000EF2A0310C10DC20DC30DCC03E72ACD1FB6
:1005E000C3134108C4004C08C1004308CC004208B2
:1005F000C3004C08C200E2294030CB00A0018316A2
:10060000811307309C009F003F30870083128A01CE
:1006100004200730A3000130A600A7008A0123218F
:10062000CC308A01EC2044308A01EC200730A30052
:100630000130A600A7008A012321CC308A01EC20DA
:10064000BE308A01EC200730A3000130A600023042
:10065000A7008A010421CE008A010421CF008A016B
:1006600020214E08C1004F08C2008A01A42244087C
:10067000D3004308D2004208D1004108D0005308FB
:10068000D7005208D6005108D500043050028A1114
:100690000A1203184D2B4B150030D400FC304F02CA
:1006A0008A110A12031C872B8A110A12031D5E2B62
:1006B0008F304E028A110A12031C872B5308BC008C
:1006C0005208BB005108BA00043050028A110A12C5
:1006D00003186C2B4B150030B900E130C800FE3018
:1006E000C7007F30C6008A30C5003C08C4003B0804
:1006F000C3003A08C2003908C1008A01E621440853
:10070000D7004308D6004208D5004108D400803005
:10071000A1008A010E2002308A019C2003308A0148
:100720009C2004308A019C2007308A019C204130A3
:100730008A019C203D308A019C205708BC00560845
:10074000BB005508BA005408B90001308A011520D1
:1007500008308A019C200330A500B4308A0137217B
:100760008A01092B8A01B22B4300200020002000BF
:0607700020002000000043
:02400E00323F3F
:00000001FF
